:103800000C942A1C0C94451C0C94451C0C94451CCF
:103810000C94451C0C94451C0C94451C0C94451CA4
:103820000C94451C0C94451C0C94451C0C94451C94
:103830000C94451C0C94451C0C94451C0C94451C84
:103840000C94451C0C94451C0C94451C0C94451C74
:103850000C94451C11241FBECFE5D4E0DEBFCDBFC4
:1038600010E0A0E6B0E0E6EEFCE302C005900D92A9
:10387000A036B107D9F710E0A0E6B0E001C01D9274
:10388000A33EB107E1F70C945D1C0C94001C81E48D
:103890000E94401E86E50E94401E82E50E94401E56
:1038A00082E40E94401E8FE40E94401E8FE40E942A
:1038B000401E84E50E94401E0895CFE5D4E0DEBF9F
:1038C000CDBFC0E0D0E001E005BF82E085BF60E091
:1038D0008BE090E00E94361E8FEF8BBBCF9B07C022
:1038E0001BBA81E085BF15BEFE0109950FC00E947D
:1038F000551E8B3141F40E94551E8335E1F70E941D
:10390000471C00E003C08FE30E94401E002331F7F4
:103910000E94551E682F813611F489E5C3C0813499
:10392000A9F40E94551E99279093E1008093E0002E
:10393000182F00270E94551E9927082B192B000FBE
:10394000111F1093E1000093E00052C0823641F451
:1039500089E50E94401E80E00E94401E80E8A2C0CF
:10396000823489F40E94551E9927182F00270E943F
:10397000551E9927082B192B0E94551E682FC80128
:103980000E94551D8FC0873689F40E94551E9927C5
:10399000182F00270E94551E9927082B192B0E94CB
:1039A000551E682FC8010E94F41DB2CF853611F54F
:1039B0008091E2008537C1F41092E1001092E0009E
:1039C00020E030E083E0F90180935700E89507B6E6
:1039D00000FCFDCF20583F4F88E32030380790F39C
:1039E0003093E1002093E00081E180935700E89557
:1039F0008DE058C0853451F488E190E028E00FB69E
:103A0000F894A89581BD0FBE21BDF2CF803581F31A
:103A10008C3471F3803711F483E544C0863421F48B
:103A200069E080E090E005C0823731F469E081E030
:103A300090E00E94691E36C08E3421F469E083E074
:103A400090E0F7CF813569F1843729F485E70E944A
:103A5000401E80E027C08857823018F40E94551E0F
:103A6000C7CF643529F40E94551E8093E200C0CF71
:103A7000633519F40E94471C4BCF663529F480E367
:103A80000E94401E84E30EC0633741F483E00E942D
:103A9000401E84E90E94401E8EE104C06B3109F48F
:103AA00037CF8FE30E94401E33CFDF92EF92FF9219
:103AB0000F931F93CF93DF938C01D62E60E070E0BD
:103AC000EB01C05ADF4F7B010894E11CF11C601729
:103AD000710718F40E94551E01C08FEF8883B7014B
:103AE0006038710568F360E070E0C091E000D0914B
:103AF000E1008CB399279C012270307081FDF9CFD1
:103B00008091E200853709F066C0FFB6F89486E43C
:103B1000D81609F03EC04091E0005091E100DB0171
:103B2000A05ABF4F8D91282F33278D919927982F19
:103B30008827282B392B6E5F7F4F81E00901FA011E
:103B400080935700E89511244E5F5F4F025010405C
:103B500049F75093E1004093E000C07885E0FE0112
:103B600080935700E89507B600FCFDCF81E1809374
:103B70005700E8958091E0009091E1009C01207849
:103B80008217930731F020583F4F3093E100209384
:103B9000E00085E4D816D9F4FB01E05AFF4F80918C
:103BA000E0008EBB8091E0009091E100292F332747
:103BB0002FBB01969093E1008093E00081918DBB33
:103BC000E29AE19AE199FECF0150104041F7FFBE21
:103BD0008DE090E001C0C901DF91CF911F910F915D
:103BE000FF90EF90DF900895FF920F931F93CF9374
:103BF000DF93EC01FFB6F894E199FECF6534B1F4A0
:103C00008091E0008EBB8091E0009091E100292F2F
:103C100033272FBB01969093E1008093E000E09A58
:103C20008DB30E94401E219759F719C060E0809122
:103C3000E0009091E1000E94691E8C010E94401EEC
:103C4000812F99270E94401E8091E0009091E10011
:103C500002969093E1008093E000229739F7FFBE2F
:103C6000DF91CF911F910F91FF9008959C01832FB9
:103C7000992780BD29B988E18AB986E880BD089571
:103C800020E030E08CB90FB607FE0BC05E990BC088
:103C90002F5F3F4F5E9907C087E220313807C4F39A
:103CA00002C05E9BFECF5E9A089580E090E00FB662
:103CB00007FE0AC05F990AC001965F9907C027E214
:103CC00080319207CCF302C05F9BFECF8CB1992765
:103CD0000895FC0160FD60935700C895802DE39521
:063CE000C895902D089527
:0400000300003800C1
:00000001FF
